:100000000EC0189518951895189518951895189567
:1000100018951895189518951895189518958FE5B1
:100020008DBFC0E4E0E44E2E81E08EBFD1E0F1E070
:100030005F2EEEEFF0E0A0E6B0E0A89584B7082EC2
:10004000877F84BF88E1992781BD91BD88278D93E3
:100050003197E9F7662480E387BB87E088BBBB98CC
:10006000AFE6B0E09C9197FF04C0B3990EC09F77B4
:100070009C93B39B0AC088E29F93992797D39F9143
:10008000B39B03C090689C93DBD281E090E08ED359
:10009000E1E0F0E0ACE6B0E091E0C2D300916C00AA
:1000A0000E3C08F005C085B78F7E806385BF8895BC
:1000B00001D0EBCF80E080936A0080E080936900FC
:1000C000ADE6B0E082D3A1E6B0E081D380E08093DA
:1000D0006500ADE6B0E00ED388E387BB87E088BB60
:1000E00081E090E063D381E080936000A6E3B0E01C
:1000F0000C9101FB81E00EF480E08F93A6E3B0E069
:100100000C9102FB81E00EF480E09F91892388230B
:1001100009F401C02CD182E080936000A6E3B0E036
:100120000C9100FB81E00EF480E08F93A6E3B0E039
:100130000C9101FB81E00EF480E09F9189238823DC
:1001400009F401C014D183E080936000A6E3B0E01D
:100150000C9100FB81E00EF480E08F93A6E3B0E009
:100160000C9102FB81E00EF480E09F9189238823AB
:1001700009F401C0FCD089E287BB86E188BB81E03D
:1001800090E014D384E080936000A6E3B0E00C918B
:1001900001FB81E00EF480E08F93A6E3B0E00C91C8
:1001A00002FB81E00EF480E09F918923882309F40B
:1001B00001C0DDD085E080936000A6E3B0E00C9143
:1001C00001FB81E00EF480E08F93A6E3B0E00C9198
:1001D00002FB81E00EF080E09F918923882309F4DF
:1001E00001C0C5D086E080936000A6E3B0E00C912A
:1001F00001FB81E00EF080E08F93A6E3B0E00C916C
:1002000002FB81E00EF480E09F918923882309F4AA
:1002100001C0ADD08AE287BB85E188BB81E090E078
:10022000C5D287E080936000A6E3B0E00C9100FBAC
:1002300081E00EF080E08F93A6E3B0E00C9102FB2A
:1002400081E00EF480E09F918923882309F401C0A6
:100250008ED088E080936000A6E3B0E00C9100FBB4
:1002600081E00EF480E08F93A6E3B0E00C9102FBF6
:1002700081E00EF080E09F918923882309F401C07A
:1002800076D089E080936000A6E3B0E00C9100FB9B
:1002900081E00EF480E08F93A6E3B0E00C9102FBC6
:1002A00081E00EF480E09F918923882309F401C046
:1002B0005ED08CE287BB83E188BB81E090E076D2A0
:1002C0008BE080936000A6E3B0E00C9100FB81E03E
:1002D0000EF080E08F93A6E3B0E00C9101FB81E08B
:1002E0000EF480E09F918923882309F401C03FD058
:1002F0008AE080936000A6E3B0E00C9100FB81E00F
:100300000EF480E08F93A6E3B0E00C9101FB81E056
:100310000EF480E09F918923882309F401C027D03F
:100320008CE080936000A6E3B0E00C9100FB81E0DC
:100330000EF480E08F93A6E3B0E00C9101FB81E026
:100340000EF080E09F918923882309F401C00FD02B
:1003500081E090E02BD2ADE6B0E00D911C91083E1B
:1003600053E0150710F009F001C0B3CE0895ADE6D3
:10037000B0E02BD2C39A84E690E018D2C39884E60A
:1003800090E014D200916900013009F00EC0809114
:10039000600080936A00A9E6B0E08C918F5F8C9337
:1003A00080E080936500ECD00895009169000230F0
:1003B00009F001C053C000916900033009F001C089
:1003C00070C0009160000B3009F009C0A9E6B0E0F0
:1003D0008C918F5F8C9380E08093650008950091ED
:1003E00060000C3009F039C046E65BE260E070E086
:1003F000A1E6B0E00D911D912D913C91F3D109F052
:1004000001C09FC081E080936600009166000830C3
:1004100010F009F021C0E6E6F0E0A190BB24EEEF79
:10042000FFEFAA0CBB1CAA0CBB1CEA0DFB1DA4E130
:10043000B0E094E0F5D1A1E6B0E00D911D912D91D1
:100440003C91D0D109F001C0C5C0A6E6B0E08C91C6
:100450008F5F8C9308F4D9CF74C041C000916000C5
:100460000C3009F01DC0E2E0F0E0A4E1B0E094E05F
:10047000D7D1A1E6B0E00D911D912D913C91B2D163
:1004800009F401C05EC07CD0A1E6B0E0A0D180E05C
:1004900080936500A9E6B0E08C918F5F8C930895FE
:1004A0001EC0009160000C3009F019C0EAE6F0E0CF
:1004B000A190BB24EEEFFFEFAA0CBB1CAA0CBB1C47
:1004C000EA0DFB1DA1E6B0E094E07BE798D158D09F
:1004D0008CEE93E1ADE6B0E08D939C930895A5E694
:1004E000B0E08C918F5F8C9300916500093010F023
:1004F00009F001C001C025C0A1E6B0E00D911D9139
:100500002D913C914AE050E060E070E000D1A1E61E
:10051000B0E00D931D932D933D93A1E6B0E00D91B6
:100520001D912D913C91A0E6B0E04C915527662796
:10053000772753D1A1E6B0E00D931D932D933D9302
:100540000895ABE6B0E08C918F5F8C9389E0809347
:1005500067008FE5809368001BD000916B0003302B
:1005600009F007C0ECE3F0E0CCD080E080936B00B2
:1005700007D08CEE93E1ADE6B0E08D939C930895A7
:1005800082E08093670088EC8093680001D0089532
:1005900084E690E00BD181E0809366004091670093
:1005A00000916600041710F009F013C0C39AA8E682
:1005B000B0E08C919927FAD0C398A8E6B0E08C916E
:1005C0009927F4D0A6E6B0E08C918F5F8C9308F465
:1005D000E5CF089580916C00815080936C00E1E03C
:1005E000F0E0ACE6B0E091E07BE709D180E08093F9
:1005F0006B00A1E6B0E0EBD0C3DFE2E2F0E0A8E6FA
:10060000B0E00BD100916800093010F009F001C092
:1006100003C089E08093680084EF91E0C7D0C59A59
:10062000A8E6B0E0EC91FF276CD0C598E1E0F0E0DF
:1006300068D08CEE93E1ADE6B0E08D939C93089585
:1006400084E690E0B3D081E080936600009166007C
:10065000083C10F009F00DC089E190E0A7D0B399F3
:1006600001C041C0A6E6B0E08C918F5F8C9308F486
:10067000EDCF8FEF8093680082E080936600009159
:100680006600023310F009F010C0A6E6B0E0EC916D
:10069000FF27A8E6B0E091E07BE7B1D0A6E6B0E0A6
:1006A0008C918F5F8C9308F4EACFE2E0F0E002EDEA
:1006B00014E020E030E0A0E1BB2794E07BE79FD08E
:1006C000E2E2F0E001E010E020E030E0A0E1BB2752
:1006D00094E07BE794D0B39B01C0FDCFBB9AE1E0EF
:1006E000F0E00FD04DDF8CEE93E1ADE6B0E08D93FE
:1006F0009C930895ED91FC91EF5FFF4FFC93EE9377
:10070000089588EE93E052D03197D9F7089522D01A
:1007100006D000FC01D0089528D030D00895842F51
:10072000952FA62FB72F4427552766277727F1E265
:10073000889409C020F4480F591F6A1F7B1F7695C3
:100740006795579547953795279517950795FA9586
:1007500089F708950024E89477FF02C006D06894D2
:1007600000F809D010F80124089512D04F5F5F4FB0
:100770006F4F7F4F0895E89437FF089500951095C7
:10078000209530950F5F1F4F2F4F3F4F689408956E
:10079000409550956095709508953197F1F70895BB
:1007A000689462F80895E89462F80895EF93FF93CF
:1007B000EE27E82BE92B31F0EAEFF0E03197F1F783
:1007C0000197D1F7FF91EF91089582E001C084E095
:1007D00099279D938A95E9F70895040F151F261F01
:1007E000371F089504171507260737070895E1995D
:1007F000FECFEEBB3196089591E001C092E07B37C9
:1008000051F47FB7F894F3DF8D918DBBE29AE19AB2
:100810009A95C9F77FBF7727089591E001C092E0CC
:0E082000E6DFE09A8DB38D939A95D1F7089597
:00000001FF
